:100000000C94AE020C94F5020C94F5020C94F502DB
:100010000C94ED250C94F5020C94F5020C94F50269
:100020000C94F5020C94F5020C9467200C94232098
:100030000C9416250C94F5020C94F5020C94F50220
:100040000C94F5020C94F5020C94F5020C94F50254
:100050000C94F5020C94F2240C94F5020C94F50225
:100060000C94F5020C94F5020C94F5020C94F50234
:100070000C94F5020C94F5020C94F5020C94F50224
:100080000C94F5020C94F5020C94F5020C94F50214
:100090000C94F5020C94F5020C94F5020C94F50204
:1000A0000C94F5020C94F5020C94F50205010980FC
:1000B000A101850319012AB700150126B700950192
:1000C00075108100C0050C0901A101850419012AE0
:1000D000A002150126A002950175108100C00660DE
:1000E000FF0961A1010962150026FF00952075082E
:1000F00081020963150026FF00952075089102C052
:1001000005010906A101050719E029E715002501E8
:10011000950875018102950175088101050719008F
:1001200029FF150026FF00950675088100050819AE
:10013000012905950575019102950175039101C08D
:10014000000101010101010101010202020202029A
:10015000020202030303030303030304040404046D
:100160000404050505050506060606060707070734
:100170000708080808090909090A0A0A0B0B0B0CE9
:100180000C0C0D0D0D0E0E0E0F0F0F101011111186
:100190001212131314141515161617171818191907
:1001A0001A1A1B1B1C1D1D1E1E1F2020212222236C
:1001B0002424252626272829292A2B2C2D2D2E2FAD
:1001C00030313232333435363738393A3B3C3D3EC4
:1001D0003F404142434445464748494A4C4D4E4FB3
:1001E00050515354555658595A5B5D5E5F61626475
:1001F000656668696B6C6D6F7072737577787A7B02
:100200007D7E8082838587888A8C8E8F9193959658
:10021000989A9C9EA0A2A3A5A7A9ABADAFB1B3B578
:10022000B7BABCBEC0C2C4C6C9CBCDCFD1D4D6D854
:10023000DBDDDFE2E4E7E9EBEEF0F3F5F8FAFDFFF2
:10024000165C1E001F002000210022002B0014005D
:100250001A000800150017003942040016000700B4
:1002600009000A00E1001D001B000600190005003E
:10027000E000E300E200C25C03512C0023002400F4
:100280002500260027002A001C0018000C00120080
:10029000130031000B000D000E000F00330034007E
:1002A0001100100036003700380028002C000251E1
:1002B0005000510052004F00165C1E001F0020002D
:1002C000210022002B0014001A0009001300050071
:1002D000394204001500160017000A00E1001D0055
:1002E0001B00060007001900E000E300E200C25C0A
:1002F00003512C00230024002500260027002A009B
:100300000D000F0018001C00330031000E0011001A
:1003100008000C001200340010000B0036003700FB
:10032000380028002C0002515000510052004F00AC
:100330003A003B003C003D003E003F0001004E0003
:1003400052004B00010001000100500051004F001D
:100350000100010001000100010001000100010095
:10036000010001000100C35C0100010040004100E8
:10037000420043004400450001004E0052004B0083
:1003800046004A000100500051004F0049004D0056
:100390000100010001000100010001000100AE00A8
:1003A000AB00A800AA00A9003A003B003C003D00B9
:1003B0003E003F000100C85CC95CC75C005C0100F6
:1003C0000100C65CCA5CC55C085D0100010001005B
:1003D0000100010001000100010001000100C35CF7
:1003E000010001004000410042004300440045007C
:1003F00001000100010001000100010001000052A4
:10040000015201000100010001000100C25CC55C55
:10041000C75CC95C01000100C45CC65CC85CCA5C06
:1004200000000000000000000000000000000000CC
:10043000000000007E0F00D4FFFFFFC7000000781F
:1004400000000000000000002A2B2800000000002F
:100450000000000000000000000000290000000073
:100460002C1E3420212224342627252E362D3738E1
:10047000271E1F202122232425263333362E3738EA
:100480001F0405060708090A0B0C0D0E0F101112A8
:10049000131415161718191A1B1C1D2F3130232D74
:1004A000350405060708090A0B0C0D0E0F10111272
:1004B000131415161718191A1B1C1D2F3130354C23
:1004C00009025B00030100A03209040000010301DE
:1004D00001000921110100012240000705810308E4
:1004E000000A0904010002030000000921110100B3
:1004F00001222200070582032000010705030320D3
:10050000000109040200010300000009211101009B
:10051000012232000705840320000A1201100100A5
:1005200000000835350235010001020301040330E3
:1005300000000014035A00790067006F006D006F1F
:100540000072007000680000000C03520047004277
:10055000004B0042000000040309040011241FBEE8
:10056000CFEFDAE0DEBFCDBF04B603FE27C0809137
:10057000F7039091F803A091F903B091FA03873043
:10058000904BA740B04BD1F41092F7031092F803B0
:100590001092F9031092FA0314BE84B7877F84BFC8
:1005A0000FB6F894A89580916000886180936000F0
:1005B000109260000FBEE0E0F8E3099523E0AAE6A0
:1005C000B2E001C01D92A73FB207E1F712E0A0E040
:1005D000B1E0E8EAF0E502C005900D92AA36B10755
:1005E000D9F70E9442210C94EE270C940000E8ED0C
:1005F000F0E080818E7F80831092E2001092DA001A
:100600001092E100A0EEB0E08C9181608C9380812B
:100610008F77808319BCA7EDB0E08C918E7F8C938F
:1006200080818F7E80831092D10308952091E40011
:100630003091E50095E6A9012091EC00822F8170B0
:1006400020FF06C08091E80080FF06C080E008958A
:100650002091E80022FD1AC08091E703882389F0E9
:10066000853089F08091EB0085FD0FC02091E4007A
:100670003091E50042175307F9F29150E1F684E01A
:10068000089582E0089583E0089581E00895EF924F
:10069000FF920F931F93CF937C018B010E9416034F
:1006A000C82F811117C08091E80085FD0BC0809193
:1006B000E8008E778093E8000E941603882399F360
:1006C000C82F08C0F70181917F018093F10001508C
:1006D000110949F78C2FCF911F910F91FF90EF9047
:1006E0000895CF93FC018091E703843001F5C09118
:1006F000E900CF702091EC00922F917020FD90E8DE
:10070000C92B82E08093E9008091E80080FF0CC053
:1007100050E040E060E270E0CF010E94470380912A
:10072000E8008E778093E800CF70C093E900CF9106
:1007300008958091DF0387FF13C08091E80082FF56
:1007400006C08091E8008B778093E80004C0809118
:10075000E7038111F2CF08958091E7038823D9F34D
:100760008091E80080FFF8CF8091E8008E77ECCF91
:10077000982F9093E900242F762F50E0891731F0BD
:100780007091EC002091ED005091F00021FD07C028
:100790009F5F973071F78093E90081E00895309171
:1007A000EB003E7F3093EB003091ED003D7F3093C6
:1007B000ED003091EB0031603093EB007093EC0072
:1007C0002093ED005093F0002091EE0027FDE0CF44
:1007D00080E00895CF92DF92EF92FF920F931F93E4
:1007E000CF93DF93C8EDD0E088818F7E8883E7EDDB
:1007F000F0E080818160808384E082BF81E080932B
:10080000D10388818E7F888302EE10E0F801108288
:100810001092DA0081EEC82ED12CF6011082888168
:100820008F77888388818068888388818F7D88839B
:1008300019BC1092E7031092DE031092DD031092B0
:10084000DC0390EEE92EF12CF70180818B7F808311
:1008500088818160888342E060E080E00E94B80384
:10086000F60180818E7F8083F801808181608083A2
:10087000808188608083F70180818E7F808388817A
:1008800080618883DF91CF911F910F91FF90EF904E
:10089000DF90CF900895FC018091E5039091E603ED
:1008A00086179707A0F06115710529F49091E8006B
:1008B0009E779093E80090E06115710551F49111D5
:1008C00008C08091E80082FF34C080E00895BC0138
:1008D000F2CF8091E7038823C1F18530C1F1809187
:1008E000E80083FD30C08091E80082FDEACF80916E
:1008F000E80080FFE1CF8091F3002091F200382FD3
:100900006115710519F02830310558F091E0283053
:10091000310509F090E02091E8002E772093E8005F
:10092000CBCF81918093F100615071092F5F3F4FD0
:10093000E7CF8091E703882341F0853041F0809133
:10094000E80083FFBECF81E0089582E0089583E050
:10095000089508958091D30308952FB7F894809156
:10096000CD039091CE03A091CF03B091D0032FBFC0
:1009700008959C01FC0132969FEF80E0419146175B
:1009800051F09F3F19F4411101C0982F8F5F8630BD
:10099000A9F79F3F09F40895290F311D97FD3A9556
:1009A000F901628308958091A10381111092A1033E
:1009B00008958091A00390919F03892B90919E03AD
:1009C000892B80936A029091A103992391F0892B3E
:1009D00080936A0220E08CE692E0FC013191CF0125
:1009E00031112F5FF2E082379F07B9F721110E9482
:1009F000D304E091B403F091B503309731F0028055
:100A0000F381E02D8AE692E009940895E92FEE0F34
:100A1000E90FEE0F8E0F982F977086958695869525
:100A200025E0829FF0011124EB58FC4F50E040E09C
:100A300080E0219130E0092E02C0369527950A9476
:100A4000E2F721703327042E01C0220F0A94EAF73F
:100A5000822B4F5F5F4F4530510559F70895E92FBD
:100A6000EE0FE90FEE0F8E0F982F977041E001C047
:100A7000440F9A95EAF786958695869595E0899F25
:100A8000F0011124EB58FC4F30E020E070E0519170
:100A9000DF011197CB01022E02C0969587950A942B
:100AA000E2F7817081958527842385278C932F5FBA
:100AB0003F4F2530310559F7089580917403909187
:100AC0004303981301C008958F5F8770FACF88237E
:100AD00041F080959091A00389238093A0030C940A
:100AE000D9040895882339F09091A003982B90930E
:100AF000A0030C94D90408952091390330913A034E
:100B00002817390771F090933A0380933903E091E5
:100B1000B403F091B503309721F00084F185E02D06
:100B20000994089520913703309138032817390725
:100B300071F09093380380933703E091B403F09100
:100B4000B503309721F00680F781E02D09940895D0
:100B500010929F0310929E030E94D90490E080E0BF
:100B60000E94920590E080E00C947C056093F10374
:100B70007093F2038093F3039093F4030C94A8050D
:100B80000F931F936091F1037091F2038091F3032F
:100B90009091F4038B019C010670112722273327C3
:100BA000063011052105310529F468601F910F9168
:100BB0000C94B605677FFACF0F931F9341E050E086
:100BC00060E070E004C0440F551F661F771F8A95D0
:100BD000D2F7CB01BA016095709580959095009100
:100BE000F1031091F2032091F3033091F403602399
:100BF0007123822393231F910F910C94B60590913A
:100C00009D038095892380939D03282F277071F47D
:100C1000282F082E000C330B9217130639F08595F8
:100C2000859585950E94DC0510929D0308950F938C
:100C30001F9341E050E060E070E004C0440F551F96
:100C4000661F771F8A95D2F78091F1039091F20386
:100C5000A091F303B091F4038A019B01082B192B97
:100C60002A2B3B2BC901B8011F910F910C94B6059B
:100C70006093A2037093A3038093A4039093A503AE
:100C80000C94A8058823B1F19CEF980F913A70F469
:100C9000ECE6F2E09191891303C0DF0111971C92F9
:100CA00042E0E237F407B1F70C94D90490E2980FD0
:100CB000983088F4877021E030E0A90102C0440F29
:100CC000551F8A95E2F7CA0180959091A003892368
:100CD0008093A003E9CF9BE5980F933020F490E038
:100CE00080E00C949205885A873120F490E080E0EF
:100CF0000C947C050895CF93C82F882309F44EC027
:100D00008CEF8C0F813AF8F4ECE6F2E082E792E0A7
:100D1000DF012D91C21759F08A179B07D1F76C2F6D
:100D20008AE692E00E94B904CF910C94D9042191F3
:100D3000C21303C0DF0111971C928E179F07B9F7EA
:100D40000E94D904ECCF80E28C0F883068F4C77021
:100D500021E030E001C0220FCA95EAF78091A0039C
:100D6000822B8093A003E0CFEBE5EC0FE33040F45F
:100D7000F0E0E75DFE4F808190E0CF910C9492050A
:100D8000C85AC73158F4EC2FF0E0EE0FFF1FE45DB6
:100D9000FE4F80819181CF910C947C05CF91089575
:100DA000E091B403F091B503309721F00190F08108
:100DB000E02D099480E00895FA01811101C0FB0142
:100DC0000994E1E8F2E0818360834283339693E003
:100DD000E533F907C1F70895FC01EE0FFF1FE80F97
:100DE000F91FEF57FD4F61834083228308950C94D0
:100DF000E1060C94EC060F931F9310E0F801EE0F40
:100E0000FF1FEB54FE4F9081905797FD9195000F77
:100E1000111FF801E758FE4F05AD0052110B2003DA
:100E2000F001219FF00D112408E310E0091B1109C6
:100E300097FD139540039001419F300D1124E20F5F
:100E4000F31F9F01220F331F2E0F3F1F37FF02C0DA
:100E500021583F4F220F232F221F330B620F1F9168
:100E60000F9108950F931F93522F10E0F801EE0F8A
:100E7000FF1FE758FE4FA5ADA052BB0B9D015203CB
:100E8000F001539FF00D1124000F111FD801AB5436
:100E9000BE4F0C910057110B40039001419F300D44
:100EA00011242E0F3F1F37FF02C0215C3F4F96E0F9
:100EB000359527959A95E1F7620F1F910F91089547
:100EC0000F931F93522F10E0F801EE0FFF1FE7580A
:100ED000FE4FA5ADA052BB0B9D015203F001539FE5
:100EE000F00D1124000F111FD801AB54BE4F0C910F
:100EF0000057110B40039001419F300D11242E0F1C
:100F00003F1F37FF02C021583F4F220F232F221FC0
:100F1000330B620F1F910F910895EF920F93972F4C
:100F200023E0029FB0011124759567956E0D792F0E
:100F30000F91EF900895322F50E0FA01EE0FFF1F4E
:100F4000E758FE4F95AD905297FD9195440F551F70
:100F5000FA01EB54FE4F2081231B330B290F311D67
:100F600097FD3A95620F0895E42FF0E0EE0FFF1F12
:100F7000E758FE4F65AD621B0895E42FF0E0EE0FD9
:100F8000FF1FEB54FE4F6081621B0895622F08958E
:100F9000E42FF0E0EE0FFF1FEB54FE4F408134EEE4
:100FA000439F412D1124E82FF0E050E0445E5F4F55
:100FB000DA01A21BB1099D01B7FF03C0319521954C
:100FC000310993E0220F331F9A95E1F7AF01421BDD
:100FD000530B9A0157FD20E0582F259F212D1124F6
:100FE000822F0895E42FF0E0EE0FFF1FEB54FE4F29
:100FF000408134EE439F412D1124E72FF0E050E073
:10100000445E5F4FDA01A21BB1099D01B7FF03C027
:1010100031952195310993E0220F331F9A95E1F71D
:10102000AF01421B530B9A0157FD20E0279F212D52
:101030001124722F0895FC019B01009729F480E090
:1010400077FF2BC080E80895AC0197FF04C04427C8
:101050005527481B590BB901640F751F37FD10C088
:10106000241B350BC901A5E0880F991FAA95E1F74C
:101070000E94A02680E2861BF7FF0FC0819508958D
:10108000CB0165E0880F991F6A95E1F7BA01621BF1
:10109000730B0E94A02680E6EECF0895EF920F9387
:1010A000CF93DF93D72FC82FC9010E19BA010E9421
:1010B0001B08602F681B7D2F8C2FDF91CF910F9124
:1010C000EF9008950F93CF93DF93D72FC82FC901C7
:1010D000BA010E941B08682F600F7D2F8C2FDF91B3
:1010E000CF910F910895EF920F931F93CF93DF93BA
:1010F000D62FC72F182FC9010E19010FBA010E9450
:101100001B08081B202F219F212D1124822F6D2FBA
:101110007C2FDF91CF911F910F91EF900895EF9267
:101120000F931F93CF93DF93D62F172FC82FC9018B
:101130000E19070FBA010E941B08702F781B719FB0
:10114000712D11246D2F8C2FDF91CF911F910F9155
:10115000EF9008950F931F93CF93DF93D62FC72F50
:10116000182FC901212F201B022FBA010E941B0832
:10117000982F990F990F891B800F282F219F212DC0
:101180001124822F6D2F7C2FDF91CF911F910F9112
:1011900008950F931F93CF93DF93D62F172FC82F48
:1011A000C901272F201B022FBA010E941B08982F6C
:1011B000990F990F782F791B700F719F712D112442
:1011C0006D2F8C2FDF91CF911F910F910895E82FF4
:1011D00086FDE0952E2F2F7086FD2F5FE695E69514
:1011E000E695E670F0E0EF5DFE4F9181929F902DC5
:1011F000212D112492959F702295207F922B208182
:10120000920F87FD919580E8890F0895AC01823097
:10121000910508F408959FEF413E8EE1580740F490
:101220009A0195E0369527959A95E1F798E0920F07
:1012300061E0E62FE90FFF27FF1F9F0135952795F6
:10124000822F229FF001239FF00DF00D11244E17E5
:101250005F0738F49FEF920F961758F78FEF860FBE
:1012600008952F3FE9F361E0620FF6CF0F93CF931C
:10127000DF93D72FC82F47FD419588E390E0841B6B
:10128000910947FD9395889FB001899F700D700D5E
:101290001124229FC001239F900D900D1124860FD1
:1012A000971F0E940609982F990F890F682F600FCA
:1012B0007D2F8C2FDF91CF910F91089530E020E0AA
:1012C000869F212D969F200D311D1124C90108955F
:1012D000AF92BF92CF92DF92FF920F931F93CF9363
:1012E000DF93362F472FE82FF0E0E05CFE4F7111BF
:1012F0000DC06491762F862FDF91CF911F910F91B2
:10130000FF90DF90CF90BF90AF900895C72FD0E0AF
:101310002491F22E022F10E056E0659FC0011124A7
:10132000EFEFF0E0BF010E948C26832F90E0880F42
:10133000991F35E5369FD001379FB00D11248A1BC8
:101340009B0B982F990F980F6F01CC1ADD0AC09E46
:10135000D001C19EB00DD09EB00D11248B2F949F53
:10136000A0011124452F55276F01C41AD50AC09E2C
:10137000A001C19E500DD09E500D11245F01A91AED
:10138000B108AC9E6001AD9ED00CBC9ED00C112467
:10139000CD2CDD24EC19FD09E09FE001E19FD00D8B
:1013A000F09FD00D1124ED2F62307105A1F048F4AB
:1013B0006115710569F06130710589F0EB2F852F9A
:1013C00007C06430710571F088F066307105B1F7BF
:1013D0006E2F722F91CFE22F2B2F8D2FF9CFE22F6F
:1013E000252FF6CFEB2F822F2D2FF2CF2B2F8F2DE6
:1013F000E52FEECF9F92AF92BF92CF92DF92EF9206
:10140000FF920F931F93CF93DF936C01C0911B0149
:101410008CE0C89FC02D11241CE01C0FB12E1D3381
:1014200010F03CE3B32E6091F003669566958091D1
:10143000E8039091E9030E945E09F82E80E48F0D85
:101440000E94E70890E8A92EA80E8F2D0E94E708B9
:1014500020E8922E980ED0E0CB1580F081E01C336E
:1014600008F080E0DF91CF911F910F91FF90EF90F6
:10147000DF90CF90BF90AF909F900895FE01E35D05
:10148000FD4F808190911C018923A1F06091ED03B3
:101490007091EE038091EF03EF2C0C2F292D4A2D34
:1014A000F60109950E946809462F282F672FCE0163
:1014B0000E94F9062196D0CF5F926F927F928F9211
:1014C0009F92AF92BF92CF92DF92EF92FF920F93D3
:1014D0001F93CF93DF933C01C0911B018CE0C89F09
:1014E000C02D11241CE01C0FF12E1D3310F03CE325
:1014F000F32E6091F00366958091E8039091E903E3
:101500000E945E09582ED0E0CE01880F991F9C01E1
:1015100027583E4F6901CF15A0F081E01C3308F039
:1015200080E0DF91CF911F910F91FF90EF90DF90BE
:10153000CF90BF90AF909F908F907F906F905F9073
:101540000895FE01E35DFD4F808190911C01892388
:1015500079F1F60184AD282F2057330B590185AD61
:10156000E82FE052FF0B4F01AA9C9001AB9C300D7D
:10157000300D1124EE9FC001EF9F900D900D1124AE
:10158000820F931F0E940609082F6091ED0370914E
:10159000EE038091EF03E52C9401A501F301099579
:1015A0000E946809462F282F672FCE010E94F90656
:1015B000F2E0CF0ED11C2196AECFAF92BF92CF9268
:1015C000DF92EF92FF920F931F93CF93DF936C0103
:1015D000C0911B018CE0C89FC02D11241CE01C0F82
:1015E000B12E1D3310F03CE3B32E6091F0036695ED
:1015F0008091E8039091E9030E945E09A82ED0E053
:10160000CE01880F991F9C0127583E4F7901CB15B9
:1016100078F081E01C3308F080E0DF91CF911F91DA
:101620000F91FF90EF90DF90CF90BF90AF90089513
:10163000FE01E35DFD4F808190911C018923C1F083
:10164000F70125AD2052330B44AD4057550B609147
:10165000ED037091EE038091EF030A2DF6010995D9
:101660000E946809462F282F672FCE010E94F90695
:10167000F2E0EF0EF11C2196CACFDF92EF92FF92BB
:101680000F931F93CF93DF937C01C0911B018CE0DC
:10169000C89FC02D11241CE01C0F012F1D3308F022
:1016A0000CE36091F003669566958091E803909154
:1016B000E9030E945E09D82ED0E0C01760F081E0F7
:1016C0001C3308F080E0DF91CF911F910F91FF90C4
:1016D000EF90DF900895FE01E35DFD4F80819091D2
:1016E0001C01892391F06091ED037091EE038091CC
:1016F000EF032D2D4C2FF70109950E946809462F05
:10170000282F672FCE010E94F9062196D6CF9091FF
:10171000B20392FF06C0282F28712830F9F4877F82
:10172000846093FF06C0282F28712831F1F4877E4A
:1017300084612091B30320FF06C0382F3871383000
:10174000D9F4877F816021FF06C0282F28712831B6
:10175000D1F4877E816194FD877E0895282F2471BE
:101760002430F9F68B7F8860DCCF282F2471243158
:1017700001F78B7E8861DDCF382F3171313019F759
:101780008E7F8860E0CF282F2171213121F78E7E56
:101790008861E1CFCF93DF9300D00F92CDB7DEB752
:1017A0009091E703943011F589837B836A8390934A
:1017B000E9008FEF9091E800815095FD06C095ED0E
:1017C0009A95F1F700008111F5CF8091E80085FF2F
:1017D0000DC050E040E063E070E0CE0101960E9451
:1017E00047038091E8008E778093E8000F900F9078
:1017F0000F90DF91CF9108952091E703243021F4D9
:10180000BC0184E00C94CA0B0895BC0183E00C94E5
:10181000CA0BCF93DF93EC018091E703843039F555
:1018200081E08093E9008FEF9091E800815095FD71
:1018300006C095ED9A95F1F700008111F5CF8091E2
:10184000E80085FF14C050E040E068E070E0CE01A1
:101850000E9447038091E8008E778093E80088E03B
:10186000FE01A4EDB3E001900D928A95E1F7DF91BE
:10187000CF91089581E08093E00080E28093D800CA
:101880001092C9008FE19EE40197F1F700C00000BB
:1018900087E090EBDC018093F7039093F803A0932B
:1018A000F903B093FA0388E19CE00FB6F894A89589
:1018B000809360000FBE90936000FFCFCF93C82F3E
:1018C0000E947B06C93349F42FEF87EE93E0215045
:1018D00080409040E1F700C000008C2FCF910C9425
:1018E00042061F93CF93DF93C62FD42F122FFC01F4
:1018F0008281882399F060933B030E94AD0490930A
:10190000360380933503C77081E001C0880FCA9504
:10191000EAF7DF91CF911F910C94720580913B0300
:10192000861340C020913503309136039FB7F89459
:101930004091CD035091CE036091CF037091D003BD
:101940009FBF421B530B483C510560F5C0E2CD0FD1
:101950008D17C1F090E2980F983048F4877091E0AD
:1019600001C0990F8A95EAF7892F0E946705C83050
:1019700048F481E09D2F977001C0880F9A95EAF78F
:101980000E947205812F0E945E0CC83090F4D770BF
:1019900081E001C0880FDA95EAF7DF91CF911F91BE
:1019A0000C946705C77081E001C0880FCA95EAF7FB
:1019B000F4CFDF91CF911F910895279A35B13F77EA
:1019C00025B120684FB7F89481E892E0FC0151916D
:1019D000CF0168E025B9000000C057FF35B9550FA9
:1019E000000000C000C000C035B900C06A9591F782
:1019F000F3E085339F0751F74FBF8FE594E00197E0
:101A0000F1F700C00000089580918002811111C09B
:101A10008091D80080618093D8008AE18A95F1F79F
:101A200000C09091D900892F817090FF82E080934F
:101A3000800281E090918002913009F080E0089569
:101A4000CF9384E090E00E944927C82F81E290E084
:101A50000E944927982F8C2FCF9108950F931F93A1
:101A6000CF93DF93C42FD0E0CC0FDD1F2CE0629F1B
:101A7000C00DD11D112438E7839FC00DD11D112445
:101A8000CE0186960E944927082F10E0102F0027CC
:101A9000CE0187960E9449279801282BC901DF9122
:101AA000CF911F910F910895462F843038F47A30EA
:101AB00028F4663018F4672F0C942E0D90E080E027
:101AC0000895CF93DF930E94540DEC018238910565
:101AD000A9F1D8F58133910509F496C048F589320A
:101AE000910509F48AC08A9709F495C0C11522E5C9
:101AF000D20708F0B6C0C11531E5D30708F026C1FA
:101B0000C83ED10508F09CC0C03ED10560F5C83A7A
:101B1000D10508F087C0C53AD10508F0EFC0C13043
:101B2000D10509F12097F9F0C430D105E0F440C0A7
:101B30008533910509F45AC0C997C1F68091B20363
:101B4000837089F0C0EED0E00EC0833E910599F11C
:101B500070F4803E910501F1823E910539F6809145
:101B6000B20382FD21C0CE01DF91CF910895863E60
:101B7000910561F1873E910571F1843E910509F06F
:101B8000B5CF8091B30381FFEECF8091B203C7EE52
:101B9000D0E084FD0DC0E7CF8091B20380FD07C186
:101BA0009091B30390FFDFCFC3EED0E084FFDBCF93
:101BB000D0E0C0E0D8CF8091B20382FDFBC090910D
:101BC000B30390FDBFCF84FFCECFF2CF8091B2039D
:101BD00083FDDDCFC8CF8091B20383FDEEC090912D
:101BE000B30391FFF0CFC4EED0E0BDCF8091B2033C
:101BF00085FFB9CFC9E2D0E0B6CF8091B20385FFAF
:101C0000B2CFC5E3D0E0AFCF8091B20386FFABCFB8
:101C1000CAE2D0E0A8CF8091B20386FFA4CFC1E38F
:101C2000D0E0A1CFCF3BD10518F6C85AD0E0CC0FF9
:101C3000DD1FC45DDE4F0990D881C02DD46493CFE1
:101C4000C11540E5D40708F064C0C11580E4D80789
:101C500008F05CC0CE019A9581159F4108F483CFAE
:101C6000A7CFC11536E5D30718F5C11545E5D4074B
:101C700008F084C0C11584E5D80708F07AC09C2F0D
:101C8000969596959E0123703327C115D34508F488
:101C900062C0C1E0D0E002C0CC0FDD1F2A95E2F7A0
:101CA00030E2939FC0011124C82BD92BDA685BCF97
:101CB000C1158AE5D80778F4C11599E5D90708F068
:101CC00068C0C11528E5D20708F472CFDC2FCC27F5
:101CD000C06FD06A48CFCE0190568115904208F06F
:101CE00067CF8D2F8F710E94870B90E0982F8827E8
:101CF00088279F719C012C2BE90149C0C55AD0E06F
:101D0000C75DDE4FC881D0E0D0642DCFDF70D06AD0
:101D10002ACFCE01E4E096958795EA95E1F78370A6
:101D20002C2F26952695237040E2249F90011124A4
:101D3000382B8C2F8370C1E0D0E002C0CC0FDD1FA8
:101D40008A95E2F7C22BD32BDC680DCFDC2FCC2792
:101D5000C16FD06A08CFC1E0D0E002C0CC0FDD1F58
:101D60002A95E2F720E2929FC0011124C82BD92BBB
:101D7000EBCFDC2FCC27C46FD06AF5CE8C2F0E941E
:101D8000870BC82FD0E0DC2FCC27CC27DF71D062A7
:101D9000EACE8C2F8F700E94870B34E0D695C795C2
:101DA0003A95E1F7CF709C2FEC01D069DCCEC9E306
:101DB000D0E0D9CEC2EED0E0D6CEC6EED0E0D3CEC3
:101DC000BF92CF92DF92EF92FF920F931F93CF9328
:101DD000DF938C01C090F103D090F203E090F30305
:101DE000F090F4038091A2039091A303A091A40327
:101DF000B091A503C82AD92AEA2AFB2ACFE1D0E06C
:101E0000BC2ED701C6010C2E04C0B695A795979598
:101E100087950A94D2F780FD0EC0219788F7B12CE0
:101E20008B2DDF91CF911F910F91FF90EF90DF905D
:101E3000CF90BF900895B8018C2F0E94610D01973B
:101E400061F3EECFCF93DF93EC010E94E00EBE0171
:101E5000DF91CF910C94610D0E94220F292F2F70DA
:101E600092959F7092509E3078F4E92FF0E0E05107
:101E7000F84D0C94B426803F19F020F4883E20F4ED
:101E800081E00895843FE1F380E00895883EC0F347
:101E9000813FD1F7F5CF822F869586958695089557
:101EA0006F927F928F929F92AF92BF92CF92DF926A
:101EB000EF92FF920F931F93CF93DF9380E4C82E8E
:101EC00082E0D82E9AEAE92EF12CE701C857D10911
:101ED00036011BC0F50185909490692DC8010E94C0
:101EE0006727682DC80101960E94672782E0A80E27
:101EF000B11C0E5F1F4FC017D10761F78CE0680E51
:101F0000711C2C96CE15DF0529F08E010C5011099D
:101F10005301E0CF7E0188E7E80EF11C88E7C80E88
:101F2000D11C8AE8E81682E0F80679F6DF91CF91B5
:101F30001F910F91FF90EF90DF90CF90BF90AF90E7
:101F40009F908F907F906F900895CF93DF93C6E01E
:101F5000D2E060E0CE010E9467272196C11584E09F
:101F6000D807B9F7DF91CF910895CF93C82F6FEFBE
:101F7000811160E282E290E00E9467276FEFC11159
:101F800067E083E290E00E9467276FEFC11163E191
:101F900084E290E0CF910C9467276CEE7EEF90E0A6
:101FA00080E00E94852760E082E090E00E94672741
:101FB00060E083E090E00E9467271092A2031092F5
:101FC000A3031092A4031092A50360E084E090E0C4
:101FD0000E94672760E081E290E00E94672760E04E
:101FE00085E090E00E94672760E086E090E00E9434
:101FF00067276FEF87E090E00E94672740E050E09E
:10200000BA0188E090E00E94792760E08DE090E0DE
:102010000E94672740E050E0BA0188E190E00E940A
:10202000792760E087E190E00E94672740E050E078
:10203000BA018CE190E00E94792760E080E290E0B4
:102040000E94672740E050E0BA018FE090E00E94D4
:10205000792740E050E0BA0183E190E00C947927C1
:102060001092A003ECE6F2E086E0DF011D928A9573
:10207000E9F70C94A8051F93CF93DF93CDB7DEB794
:10208000AA970FB6F894DEBF0FBECDBF8FED93E0D9
:102090002091F100DC012D93CD01B3E0873E9B0739
:1020A000B9F78091E003833009F471C0B8F481304E
:1020B00009F448C0823009F4B2C08091E80083FF7F
:1020C00093C28091DF039091E0039A3008F08CC2B4
:1020D000E92FF0E0E250F84D0C94B4268A3009F470
:1020E0008DC08B3009F470C0893039F78091DF03DF
:1020F000813219F78091E3039091E403009711F086
:102100000297D9F68091E800877F8093E80080915C
:10211000E80082FF37C09091F3008091F2000297AF
:1021200029F48091F1008B7F813021F48091F100BE
:102130008093D3038091E8008B778093E8000E941E
:102140009903BBCF8091DF03813A09F0B6CF80912C
:10215000E800877F8093E8008091E3039091E40397
:10216000892B61F468E084ED93E070E00E944B04F9
:102170008091E8008B778093E8009FCF60E090E04B
:1021800080E0F3CF8091E7038111C1CF96CF80919A
:10219000DF03813A09F091CF8091E3039091E4034A
:1021A000892B09F08ACF8091E800877F8093E8002F
:1021B0008091E80080FFFCCF80911A018093F100AC
:1021C0008091E8008E77B9CF8091DF03813209F0EA
:1021D00074CF8091E3039091E403892B09F06DCFD4
:1021E0008091E800877F8093E8000E9499038091A6
:1021F000E10380931A010E9430105FCF8091DF03CA
:10220000813209F05ACF8091E800877F8093E800FF
:102210000E9499038091E2038093D2034ECF809174
:10222000DF03813A09F049CF8091E800877F8093EE
:10223000E8008091E80080FFFCCF8091D203BECF00
:10224000803899F0823809F0CFC18091E3038F7014
:10225000873008F0C9C18093E9008091EB0085FBCD
:10226000882780F91092E90006C08091DC039091E4
:10227000DD03911182609091E800977F9093E800D0
:102280008093F1001092F1008091E8008E77A8C150
:10229000882309F496C1823009F0A6C18091E10338
:1022A000811199C18091E3038F702FEF280F2630A1
:1022B00008F09AC18093E9002091EB0020FF8BC1C8
:1022C000933031F48091EB0080628093EB0083C106
:1022D0009091EB0090619093EB0021E030E001C021
:1022E000220F8A95EAF72093EA001092EA00809183
:1022F000EB008860EACF811177C11091E1031F776D
:102300008091E3008078812B8093E3008091E80046
:10231000877F8093E8000E9499038091E80080FF06
:10232000FCCF8091E30080688093E30082E011118C
:1023300083E08093E70358C18058823008F054C18D
:102340002091E1033091E2032C3DE3E03E07A1F54B
:1023500083E08A838AE289834FB7F894DE0113967B
:1023600020E03EE051E2E32FF0E050935700E4918B
:1023700020FF03C0E295EF703F5FEF708E2F90E07B
:10238000EA30C0F0C7968D939D932F5F243159F7A3
:102390004FBF8091E800877F8093E8006AE270E099
:1023A000CE0101960E944B048091E8008B778093C8
:1023B000E8001AC1C096E7CF8091E3039091E4034F
:1023C000432F55274330510509F44AC078F5413071
:1023D000510509F485C08BE590E0E0ECF4E0423073
:1023E000510509F001C12091E800277F2093E80002
:1023F0002091E5033091E6038217930708F49C01CE
:1024000040E02115310509F070C041116EC0809186
:10241000E80082FDC9CF8091E703882329F2853047
:1024200019F28091E80083FFF2CFBECF413251050F
:1024300009F447C04232510509F0D6C083309105F6
:1024400008F0D2C0FC01EE0FFF1FE359FE4F0190D0
:10245000F081E02D86599E4FDC018C9190E01DC0EB
:10246000332721303105E9F02115310579F022308B
:102470003105F9F02330310509F0B6C0EDE2F5E0A1
:10248000E4918E2F90E0EDE2F5E007C0E7E5F5E09E
:10249000E4918E2F90E0E7E5F5E0009709F4A4C001
:1024A000A2CFE9E4F5E0E4918E2F90E0E9E4F5E0D5
:1024B000F4CFE3E3F5E0E4918E2F90E0E3E3F5E081
:1024C000ECCF8330910508F08FC0880F991FFC0175
:1024D000ED58FE4F0190F081E02D89E090E083CF30
:1024E00082E190E0EBE1F5E07ECF8091E703882385
:1024F00009F45ACF853009F457CF8091E80083FD65
:1025000053CF8091E80082FD82CF8091E80080FF68
:1025100078CF9091F3008091F2002115310519F0E8
:102520008830910550F041E0089709F040E0809133
:10253000E8008E778093E80064CF44914093F100E7
:102540003196215031090196E8CF803809F04CC00E
:102550008091E800877F8093E8008091DE0380937C
:10256000F10092CE811140C01091E1031230E0F5EC
:102570008091E800877F8093E8001093DE030E943B
:102580009903112311F084E005C08091E30087FDD9
:10259000FACF81E08093E70342E061EC81E00E94A2
:1025A000B80342E261EC84E00E94B80342E261ECCD
:1025B00082E00E94B80342E260EC83E00E94B8032C
:1025C00013C08091E103813079F481E0933009F008
:1025D00080E08093DD031092E9008091E800877F1E
:1025E0008093E8000E9499038091E80083FF0AC06D
:1025F0008091E800877F8093E8008091EB00806203
:102600008093EB00AA960FB6F894DEBF0FBECDBF45
:10261000DF91CF911F9108951F93CF93DF93EC012A
:10262000FC01E35DFD4F80816823A1F00E94292712
:10263000182F0E942927612F782F8091EF030E9485
:102640006809462F282F672FCE01DF91CF911F9168
:102650000C94F906DF91CF911F910895DF92EF92CC
:10266000FF920F931F93CF93DF938C01FC01E35DE7
:10267000FD4F8081682381F1D090EE03D091EF036C
:10268000C091ED03EC2EF12C0E942927282FC701C1
:102690008C549F4F68E671E00E94A0268E199F0916
:1026A00097FD0396959587959595879523706C2F43
:1026B000289F600D11247D2D8D2F0E946809462FC3
:1026C000282F672FC801DF91CF911F910F91FF90A5
:1026D000EF90DF900C94F906DF91CF911F910F914D
:1026E000FF90EF90DF90089545E050E06CE170E0DE
:1026F0008CEE93E00C9457278091EC03982F9695DD
:1027000096959F5F9F738370993148F4990F990F45
:10271000892B8093EC0310920F010C947413846046
:10272000F8CF8091EC0384508093EC03982F9C7F2A
:1027300021F4837080668093EC0310920F010C9457
:102740007413ECEEF3E08181885F81830C94741341
:10275000ECEEF3E08181885081830C947413ECEEED
:10276000F3E0228130E1230F08F42FEF22830C9451
:102770007413ECEEF3E0228130E1231B08F420E037
:1027800022830C9474132091EF0330E1230F08F49B
:102790002FEF273920F42093EF030C94741386E96C
:1027A0008093EF03FACFECEEF3E0238130E1231BBB
:1027B00008F420E023830C947413ECEEF3E02481FE
:1027C00030E1230F08F42FEF24830C947413ECEE04
:1027D000F3E0248130E1231B08F420E024830C94EF
:1027E00074133F924F925F926F927F928F929F925B
:1027F000AF92BF92CF92DF92EF92FF920F931F930F
:10280000CF93DF9300D000D00F92CDB7DEB77C011D
:10281000FC0183819481892B31F08081918189230E
:102820008F3F09F08CC50F900F900F900F900F9075
:10283000DF91CF911F910F91FF90EF90DF90CF909C
:10284000BF90AF909F908F907F906F905F904F90D0
:102850003F9008950E94E00E182F682F89819A8179
:102860000E942F0569817A81812F0E94540D8C016D
:10287000F7019281992309F457C5980122513F45E8
:102880002031310508F029C58FEF93E00E944927D8
:10289000025156E0852E52E0952E882381F18091D9
:1028A0009D03877009F4BFCFF7018281882309F463
:1028B000BACF82E00F900F900F900F900F90DF91A2
:1028C000CF911F910F91FF90EF90DF90CF90BF902D
:1028D000AF909F908F907F906F905F904F903F90C0
:1028E0000C94FF058114F4E09F06C9F2C4010E9414
:1028F0004927811101C001502FEF821A920A01115C
:10290000F1CF1C821B82662463944AE0542E84011A
:102910000F5F1F4FC4010E94492789831A828823B1
:1029200009F4BDCF9FEF980F933008F58A83698231
:1029300032E0830E911CC8010E9449278B838823B3
:1029400009F4ADCF8E010F5F1F4FF80120812223C4
:10295000F1F2213009F043C091818281913049F434
:102960000E5F1F4F0E945E0C0F5F1F4FEECF48019E
:10297000E9CF923029F40E5F1F4F0E947B06F4CFFF
:10298000933029F40E5F1F4F0E944206EDCF943022
:1029900019F00F5F1F4FE8CF0E5F1F4F30E020E0B0
:1029A000B8016F5F7F4FF80141818053990B8A30E6
:1029B000910550F021503109B8F28FE99FE001975D
:1029C000F1F700C00000F6CF529EF001539EF00DCB
:1029D00011249C012E0F3F1F842F8B01E1CFE22F8A
:1029E000F0E0E05CFB4F7490822F8695869586958B
:1029F00090E0FC01E05DFB4FA4902770B12C022E0B
:102A000002C0B594A7940A94E2F7E1E0AE22BB2499
:102A1000FC01E05EFB4FC490D12C02C0D594C7945A
:102A20002A95E2F7F1E0CF22DD24A114B10419F0D8
:102A300081EE0E947B06C114D10419F086EE0E943B
:102A40007B06872D0E945E0CCD2819F086EE0E9431
:102A50004206AB2809F488CF81EE96CF81E00E9430
:102A6000170603C081E00E94DC050E94C00517CF55
:102A700082E0F5CF053F2CE5120709F461C008F4A8
:102A80005BC027E245EE66EE063F8CE5180709F4C9
:102A900047C4992309F464C410923B030230ECE567
:102AA0001E0708F430C10631FCE51F0738F0980115
:102AB0002A5F3C452930310508F025C10E94200DD0
:102AC0009093B3038093B20300312CE5120709F40D
:102AD000E9C008F073C008308CE5180709F4D4C0C9
:102AE00008F045C00430ECE51E0709F4C1C078F5D4
:102AF00002302CE5120709F4B5C08091B203826060
:102B000003301C4509F4B1C06091B2031091B303C6
:102B100084E090E00E946727612F81E290E00E94AC
:102B200067270E943010BBCE27E245EE65EEF8C362
:102B300026E241EE60EEF4C327E245EE64EEF0C318
:102B400026E241EE62EEECC328E241E0EFCF063030
:102B50008CE5180709F494C08091B20388600730AF
:102B60001C4508F482C08091B20380627EC08091CF
:102B7000B2038D7F0C30ECE51E0709F476C070F4CB
:102B80008091B2038C600A302CE5120709F46DC005
:102B900008F47EC08091B2038E7F67C00E308CE552
:102BA000180709F47BC08091B2038B7F0F301C455E
:102BB00008F45BC08091B2038F7E57C00B3FECE5F9
:102BC0001E0709F459C030F503312CE5120709F44A
:102BD00071C078F401318CE5180709F467C002313F
:102BE0001C4509F091CF0E9430108091B2038F777D
:102BF0003CC00531ECE51E0709F464C008F478C058
:102C00008091B30381600A3F1C4509F07DCF80931A
:102C1000B3037ACF0F3F3CE5130709F44FC088F4A4
:102C20008091B3038D7F0D3F9CE5190781F380915F
:102C3000B3038E7F0E3F1C4550F38091B303836036
:102C4000E6CF0130FDE51F0709F45BC008F446C07C
:102C500060E002301D4509F057CF8EE090E00E9401
:102C6000672752CF8091B20381608093B2034CCF2B
:102C70008091B2038460F9CF8091B3038260C7CFA3
:102C80008091B2038061F1CF8091B2038064EDCF77
:102C90000E9430108091B2038068E7CF8091B20328
:102CA000877FE3CF8091B2038F7DDFCF8091B20326
:102CB0008F7BDBCF8091B203837FD7CF8091B3032B
:102CC0008C7FA5CF8091B20382FB992790F921E0F8
:102CD000922790FB82F990FB83F9C7CF8091B303D1
:102CE000982F909591708E7F892B90FB81F98FCFD3
:102CF0000E9430109091B203892F97FB87F980587A
:102D0000B4CF61E0AACF06318CE5180709F03AC3C9
:102D10008091A0038A7A91E009F490E090933C03BB
:102D200069E2811165E38AE692E00E94B9040E949B
:102D3000D904B5CD80913C0381110FC089E2ECE646
:102D4000F2E022E732E09191891303C0DF0111978D
:102D50001C922E173F07B9F7EACF85E3F0CF809199
:102D6000EC0391E089278093EC0310920F010E94FD
:102D7000741395CD41E953E16CE773E10E94DC06E1
:102D80008ECD4CE753E161E973E1F8CF48EA53E1B6
:102D900061EA73E1F3CF41EA53E168EA73E1EECF10
:102DA00049EB53E16FEA73E1E9CF4FEA53E169EB95
:102DB00073E1E4CF43ED53E163EC73E1DFCF43EC28
:102DC00053E163ED73E1DACF47EE53E16DED73E16B
:102DD000D5CF4DED53E167EE73E1D0CF8091EC0399
:102DE00083708460C0CF8091EC0383708461BBCF1B
:102DF0008091EC0383708463B6CF8091EC03837081
:102E00008864B1CF0E9430109FEFE4E3FCE0915062
:102E1000E040F040E1F700C000000E943A0C0E9440
:102E2000CD0F3DCDC8010E940605D82EC2C2212F6C
:102E30002F70C22E107F19F0C29490EFC922AA20E1
:102E4000C9F0CC2069F080E28B0D883010F00111C0
:102E50000BC08091A003C82AC092A0030E94D9048D
:102E60008B2D0E947B0619C080919F03C82AC092B7
:102E70009F03F4CF8B2D0E944206CC2071F0C094AA
:102E800080E28B0D883010F001113CC08091A003CE
:102E9000C822C092A0030E94D904ED2DE850FF0B78
:102EA000349710F40E94D006332009F4BCCC8091F2
:102EB0009D0380FDB8CCF701128285958595859597
:102EC0000E941706C7010E94F11380919D0385950A
:102ED000859585950F900F900F900F900F90DF9133
:102EE000CF911F910F91FF90EF90DF90CF90BF9007
:102EF000AF909F908F907F906F905F904F903F909A
:102F00000C94DC0580919F03C822C0929F03C3CF1D
:102F1000312F3F70C32E107F103219F0C29480EF12
:102F2000C822002369F0013061F1AA20B9F199208B
:102F300071F1F701858180FF93CF8F70858327C062
:102F4000AA2091F09091A1038C2D892B911003C0A0
:102F50000E947205A2CFE1E09E12FACF891709F410
:102F60009CCF8093A10399CF911006C00E94D304F7
:102F70008C2D0E94670591CFF1E09F1609F48DCF4B
:102F8000F5CFAA2031F025E0291508F486CF8C2D45
:102F9000DFCF34E0391508F480CFEACF992041F330
:102FA000093349F4FFEF27EE33E0F1502040304081
:102FB000E1F700C000008B2D0E9442066ECF812FEA
:102FC00086958695837069F0813009F066CF8B2DE8
:102FD000912F9370A11002C090E080E00E947C05C8
:102FE0005CCF8B2D912F9370A11002C090E080E0F8
:102FF0000E94920552CF812F837009F06CC0A110FE
:103000004CCF8B2D829586958770880F880F6B2DFE
:103010006F70462E512C712C612C082E04C0440C6C
:10302000551C661C771C0A94D2F740E050E0BA01A8
:10303000B4FE0FC04FE050E060E070E004C0440F09
:10304000551F661F771F8A95D2F74095509560955A
:103050007095169516951370123019F1A8F5809099
:10306000A2039090A303A090A403B090A5031130F5
:1030700069F04429552966297729CB01BA016821CD
:1030800079218A219B210E94380607CF8428952820
:10309000A628B728CB01BA01682979298A299B2952
:1030A000F2CF44295529662977298090A203909070
:1030B000A303A090A403B090A503CB01BA01682597
:1030C00079258A259B25DFCFCB01BA016429752993
:1030D00086299729D8CF8695AA2011F0812F817053
:1030E000882309F4DACE8B2D829586958770880F18
:1030F000880F6B2D6F70462E512C712C612C082E71
:1031000004C0440C551C661C771C0A94D2F740E09E
:1031100050E0BA01B4FE0FC04FE050E060E070E054
:1031200004C0440F551F661F771F8A95D2F740953C
:10313000509560957095169516951370123019F18B
:10314000A8F58090F1039090F203A090F303B09063
:10315000F403113069F04429552966297729CB01F8
:10316000BA01682179218A219B210E94B60595CE5A
:1031700084289528A628B728CB01BA01682979297F
:103180008A299B29F2CF44295529662977298090DD
:10319000F1039090F203A090F303B090F403CB01FD
:1031A000BA01682579258A259B25DFCFCB01BA0195
:1031B0006429752986299729D8CF1F70AA2029F05C
:1031C000812F0E9417068B2DC3CE8B2D0E94670581
:1031D000812F0E94DC0561CE8B2D023F09F44AC08D
:1031E00060F4003FF9F0013FE9F1AA2009F465C05D
:1031F000911036CE812F8F713AC0033F09F43FC042
:10320000043F99F7AA2009F44DC01F71812F0E9435
:103210001706E8E01E9FC0011124836080939D0380
:10322000812F25C0AA20C9F084E0891508F435CE85
:103230001F7161E070E080E090E004C0660F771FCE
:10324000881F991F1A95D2F78090F1039090F2038E
:10325000A090F303B090F403A4CF95E0991508F47F
:103260001CCEE6CF812F8F71AA2009F4B2CF0E9425
:10327000170613CE812F8F71AA20C9F3AACF60E061
:1032800070E0CB01AA2009F470CF1F7161E070E0FB
:1032900080E090E004C0660F771F881F991F1A9581
:1032A000D2F763CF81E00E94FF05F1E0F91508F045
:1032B000F4CD82E00E94FF05F0CD992059F08933CA
:1032C00009F079CE2FEF37EE83E021503040804077
:1032D000E1F76FCE812F8F717CCF0031FFE51F07A3
:1032E00009F4BCCB01312FE5120709F4C1CB033F30
:1032F0002CE5120709F41CCC08F0BCCB083D8CE58A
:10330000180709F411CC093DECE51E0709F41CCCA3
:10331000073DFCE51F0709F0BCCB26E241EE61EE5C
:10332000C7010E94710CBBCA00313FE5130709F4C5
:1033300099CB01318FE51807D1F682E094CB85E077
:10334000DE01119601900D928A95E1F7F701228135
:1033500089819A8121117ECA0E940605182F82CA8E
:103360000631FCE51F0709F4E5CC8091A0038272C9
:10337000F801E25CFC45E431F10568F4E85FF74DE3
:103380000C94B42601152CE5120709F43BCD0E3D33
:103390001C4509F444CDF70100811181992309F4FA
:1033A00041CDC8010E94E00ED82E682FC8010E94AE
:1033B0002F05B8018D2D0E94610DB82E192F082FF1
:1033C000F701958092943FE09322A280A110109281
:1033D0009F0380919D03877099F0AA2089F0812F27
:1033E000807F803421F080E28B0D883048F082E0CD
:1033F0000E94FF0580919D038770332433948111CF
:10340000312CD12ED2942FE0D222FBE0FD1508F40E
:1034100044CDED2DF0E0E45EF74D0C94B4261F93FF
:10342000CF93DF9380914203807FA9F480913F0383
:10343000882389F080917403D091430360913D0308
:1034400070913E03A0914003B0914103C62FC72362
:1034500016E0D81304C0DF91CF911F91089590E03A
:10346000109711F0CF3F19F401968770F2CF189F93
:103470009001199F300D1124F901EC5BFC4F418143
:103480004713F2CF40814613EFCF42814111ECCF79
:10349000438154814A1B5B0B483C510528F78091BE
:1034A00042038F70806180934203F901E75BFC4F18
:1034B00080818F70806180838DE393E00E94F1139F
:1034C000DF91CF911F910C945D05AF92BF92CF9287
:1034D000DF92EF92FF920F931F93CF93DF93CDB7BD
:1034E000DEB761970FB6F894DEBF0FBECDBF8C017B
:1034F00085E0F801DE011D9601900D928A95E1F7B5
:10350000F80180819181E2802DE3A22E23E0B22E8A
:1035100060914003709141036115710509F43EC14A
:1035200030913D0340913E03232F24232F3F09F484
:1035300035C1C380D480F0903F03F601E61BF70B42
:10354000FF2009F4FBC020914203522F507FE83C3A
:10355000F10508F0BBC0511178C0FE2C491321C001
:1035600038131FC0E1101DC02F702061209342034B
:10357000C5010E94F11380914203F80185838F2DCC
:1035800061960FB6F894DEBF0FBECDBFDF91CF912D
:103590001F910F91FF90EF90DF90CF90BF90AF9071
:1035A0000895CD2829F0282F29232F3F09F014C191
:1035B00020E0F22FF170DF2E20FF3DC02091740338
:1035C0004091430356E0241315C08D879E878D8557
:1035D0009E850E94220F292F22952F702230F8F00D
:1035E000243020F59F70F9F0F8019581907FD9F48F
:1035F000D12C1FC030E0529FF001539FF00D1124D9
:10360000EC5BFC4F6181961306C06081861303C09A
:103610006281E61210C02F5F3F4F2770D4CF9F709A
:1036200011F0882329F3805E883010F3C8010E94CE
:10363000F113FD2CA4CFEE2009F4A1CF8091420319
:10364000816080934203F12C9ACF491312C0381342
:1036500010C0E1100EC0F8012583C8010E94F113CB
:1036600086E0F801ADE3B3E001900D928A95E1F7B1
:1036700086CF8D879E878D859E850E942C0F8823FF
:1036800009F1EE20F9F080914203803270F0209130
:103690003D0330913E0338872F831986DB86CA8627
:1036A0008C87CE0107960E94F11386E0F801ADE306
:1036B000B3E001900D928A95E1F70E940F1AFF2462
:1036C000F3945DCFC8010E94F113F9CF51110AC0E4
:1036D0008DE393E00E94F11386E0F50111928A9543
:1036E000E9F7B1CF49130FC038130DC0E1100BC07B
:1036F000F8012583C8010E94F11386E0F5011192BB
:103700008A95E9F73CCF8D879E878D859E850E949F
:103710002C0F8823B9F2EE20A9F280914203803267
:1037200020F220913D0330913E033A8329831B828E
:10373000DD82CC828E83CE010196B5CFE83CF105C7
:10374000E0F6FE2CEE2009F4BDCF491316C0381365
:1037500014C08091420380FD83CF982F907F09F49D
:103760007FCFF8018583903F09F477CF982F907F22
:10377000905F8F70892B858370CF8D879E878D8515
:103780009E850E942C0F811190CF80914203816011
:1037900080934203C8010E94F113F1CEEE2009F498
:1037A00091CF8D879E878D859E850E942C0FF82E48
:1037B000882309F487CF86E0F801ADE3B3E00190F8
:1037C0000D928A95E1F780913D0390913E030E940E
:1037D000220F0E940F1AD3CE21E02E25EACE1F938E
:1037E000CF93DF93CDB7DEB767970FB6F894DEBF00
:1037F0000FBECDBF4B8B5C8B6D8B7E8B8F8B1A8AF4
:10380000198A85E0FE017396DE011D9601900D92E6
:103810008A95E1F786E0FE013D96DE01179601905C
:103820000D928A95E1F7CE0107960E94651A8111E3
:1038300012C086E0FE013796DE01119601900D92CE
:103840008A95E1F78A859B85892B29F08F81988558
:1038500089238F3FB1F516E0809174039091430363
:1038600089131DC067960FB6F894DEBF0FBECDBF9B
:10387000DF91CF911F91089596E0929FD001939F81
:10388000B00D1124AC5BBC4FFE01319601900D923E
:103890009A95E1F7809343030E945D05DCCF819FF9
:1038A000C00111248C5B9C4F0E94651A8823D1F2C1
:1038B0008091740390E00196877099278093740338
:1038C000CBCF2091430330E0C9010196877099273F
:1038D000409174034817190679F60E94301010922F
:1038E00043031092740386E0EDE3F3E0DF011D92E1
:1038F0008A95E9F7B0CFECEEF3E085E38083809121
:103900001E0190911F01A091200181839283A383C6
:103910008FE784830C9474136F927F928F929F929F
:10392000AF92BF92CF92DF92EF92FF920F931F93CD
:10393000CF93DF934AE551E006EA13E0EFE5AE2EC0
:10394000E1E0BE2E3801C0E0EE24E394F12CDA0170
:103950008D91AD01E82FE295EF70F0E091A18F70AD
:10396000B70101C0660F8A95EAF7892F862B81A3DC
:1039700082A1862E8094882182A3B0EABA95F1F7BD
:1039800074E6C72E71E0D72E30E020E0D0E0D601FB
:103990009D906D01892D82958F7090E0DC0190964D
:1039A0008C9190E0B92DBF7002C095958795BA951E
:1039B000E2F780FD50C08E2D022E01C0880F0A94C0
:1039C000EAF7D82B2F5F3F4F2630310501F781A151
:1039D000882281A282A1682B62A3F3018081D8177B
:1039E000E1F1D08381E0C82BFFEF6F1A7F0AA416A4
:1039F000B50609F0ACCFD091B103CC2381F181E0C1
:103A0000809375020E94AD049093740280937302B8
:103A100020917302309174024FB7F8948091CD03D6
:103A20009091CE03A091CF03B091D0034FBF821BE2
:103A3000930B0697C0F0ED2FF0E0ED53FC4F8BEAAF
:103A400093E0D8012D918D0121938A179B07C9F727
:103A50001092750208C080E0B4CF80E0C4CF80919E
:103A600075028111D5CF0E94040D882309F4DAC2B2
:103A7000D091B0030E943F26009709F440C0809186
:103A80007F028F5F80937F02863008F048C08FB737
:103A9000F8944091CD035091CE036091CF03709183
:103AA000D0038FBF409376025093770260937802E1
:103AB000709379028091EC03D82FD37019F0D82F2E
:103AC000D695D69590910F01913009F441C0992374
:103AD00089F1923009F47FC2933009F484C28C2FAB
:103AE000DF91CF911F910F91FF90EF90DF90CF90DA
:103AF000BF90AF909F908F907F906F900895ED2F23
:103B0000F0E0ED53FC4FDC01A658BD4F2C91219302
:103B1000019685309105B9F710927F02B8CFE091F8
:103B2000B003F0E0ED53FC4F108211821282138239
:103B30001482ADCF10921B014093E8035093E90328
:103B40006093EA037093EB0381E080930F01C7CF8A
:103B50009091050111E0D91309C0837020910401EF
:103B600030E011E08217130609F410E01170109391
:103B70001D01D93140F4ED2FF0E0E85DF74D0C94D4
:103B8000B426111102C010E027C040E060E080E0E0
:103B90000E94F706F8CF00911B018CE0089F002DD2
:103BA00011244CE0F42EF00EEF2CBCE3BF1510F402
:103BB0003CE3E32E6091ED037091EE038091EF03FF
:103BC0000E946809D62EC72EB82E10E00E15B0F050
:103BD00011E0EBE3EF15B8F280911B018F5F80934A
:103BE0001B0111117CCF82E080930F0180911D0198
:103BF000811175CFD11173CF83E0A7CFF801E35DB9
:103C0000FD4F808190911C01892331F02B2D4D2D8A
:103C10006C2DC8010E94F9060F5F1F4FD7CF00918E
:103C20001B018CE0089F002D11242CE0F22EF00ED9
:103C3000EF2CFCE3FF1510F49CE3E92EC090EE039B
:103C4000D090EF031091ED03612F7C2D8D2D0E94FC
:103C50006809B62EA72E982E6091F003610F7C2D77
:103C60008D2D0E946809D62EC72E882E10E00E15C5
:103C700030F011E02BE32F1508F0AECF84CFF80120
:103C8000E35DFD4F908180911C01892359F0282D1F
:103C90004D2D6C2D90FD03C0292D4B2D6A2DC80193
:103CA0000E94F9060F5F1F4FE2CF00911B018CE0CD
:103CB000089F002D11248CE0F82EF00EDF2C3CE341
:103CC0003F1510F41CE3D12EC090EE03B090EF032B
:103CD0002091F003B0E4EB2E3E2D329F312D1124C4
:103CE000E32E10E00D1530F011E08BE38F1508F096
:103CF00073CF49CFF801E35DFD4F808190911C01A6
:103D00008923B9F0F801EE0FFF1FE758FE4F85AD8C
:103D100082958F706091ED038E9D600D11247C2D36
:103D20008B2D0E946809462F282F672FC8010E94FB
:103D3000F9060F5F1F4FD6CF00911B018CE0089F43
:103D4000002D1124ECE0FE2EF00EDF2C9CE39F15DD
:103D500010F47CE3D72EC090EE03B090EF032091D7
:103D6000F00360E4E62E3E2D329F312D1124E32E28
:103D700010E00D1508F0B8CFF801E35DFD4F80812C
:103D800090911C018923D9F0F801EE0FFF1FE7582D
:103D9000FE4F64ADE69EB001112455E07595679520
:103DA0005A95E1F78091ED03680F7C2D8B2D0E94D1
:103DB0006809462F282F672FC8010E94F9060F5F58
:103DC0001F4FD7CF10911B018CE0189F102D11248D
:103DD0003CE0F32EF10EEF2C9CE39F1510F42CE346
:103DE000E22ED090ED030091EE03C090EF036091BE
:103DF000F0036695669566958091E8039091E903D6
:103E00000E945E090E94E708805887FD8195880F0F
:103E1000282F3C2D239F212D1124822F6D2D702FB3
:103E20000E946809D62EC72EB82E012F10E00E155D
:103E300008F05ACFF801E35DFD4F808190911C019D
:103E4000892331F02B2D4D2D6C2DC8010E94F906D0
:103E50000F5F1F4FECCF82EF97E00E943D0B182FB2
:103E6000BBCE88EC97E0F9CF89EC98E00E94DD0AA0
:103E7000F6CF8AEA98E0FACF8FE898E00E945C0AD1
:103E8000EECF83E798E0FACF86EC97E0E6CF8DEBB4
:103E900097E0E3CF84EB97E0E0CF8BE997E0DDCFCD
:103EA0008DE897E0EBCF86E399E0E0CF82E698E0FB
:103EB000DDCF8EE498E0E2CF80E697E00E94FA0939
:103EC000CECF82E397E0FACF8BEF96E0F7CF1111D8
:103ED0001EC06091F00320E1620F08F46FEF809143
:103EE000E8039091E9030E945E096AE070E00E9495
:103EF0008C26892B09F047CE0E9429276CE370E0BD
:103F00000E94A02660911C010E942E1365CE009194
:103F10001B018CE0089F002D11249CE0D92ED00EAF
:103F20008D2D9CE39D1508F48CE310E0E82EF12C18
:103F30000E151F0534F011E0ABE3AD1508F04CCEC3
:103F400022CE60911C01C8010E942E130F5F1F4FEB
:103F5000EFCF11111EC06091F00320E1620F08F451
:103F60006FEF8091E8039091E9030E945E0965E09C
:103F700070E00E948C26892B09F005CE0E9429272B
:103F80006CE370E00E94A02660911C010E940C135B
:103F900023CE00911B018CE0089F002D11248CE0A2
:103FA000D82ED00E8D2DBCE3BD1508F48CE310E0A7
:103FB000E82EF12C0E151F0534F011E0EBE3ED15A2
:103FC00008F00ACEE0CD60911C01C8010E940C13DC
:103FD0000F5F1F4FEFCFD0930501837080930401D3
:103FE0000E94DD0C09CE4091E8035091E9036091F5
:103FF000EA037091EB032FB7F8948091CD03909171
:10400000CE03A091CF03B091D0032FBF841B950B9B
:10401000A60BB70B4097A105B10508F460CD10922F
:104020000F015DCDE091B103F0E0ED53FC4F90E066
:1040300080E02191DC01A658BD4F2C93019685307C
:104040009105B9F74CCD1F920F920FB60F92112424
:104050002F933F934F935F936F937F938F939F9390
:10406000AF93BF93CF93DF93EF93FF93D091E9008A
:10407000DF708091EC00C82FC17080FDC0E8109205
:10408000E9008091F000877F8093F00078940E948F
:104090003B101092E9008091F00088608093F0005E
:1040A000CD2BCF70C093E900FF91EF91DF91CF91BD
:1040B000BF91AF919F918F917F916F915F914F9140
:1040C0003F912F910F900FBE0F901F9018951F9248
:1040D0000F920FB60F9211242F933F934F935F933C
:1040E0006F937F938F939F93AF93BF93EF93FF93C0
:1040F0008091E10082FF09C08091E20082FF05C04B
:104100008091E1008B7F8093E1008091DA0080FF55
:1041100024C08091D80080FF20C08091DA008E7F7B
:104120008093DA008091D90080FF9FC080E189BD33
:1041300082E189BD09B400FEFDCF81E08093E703F1
:104140008091D103811109C00E94F7020E94EA0305
:104150008091E20084608093E2008091E10080FF22
:1041600017C08091E20080FF13C08091E2008E7F33
:104170008093E2008091E20080618093E200809170
:10418000D80080628093D80019BC85E08093E70353
:104190008091E10084FF2DC08091E20084FF29C05E
:1041A00080E189BD82E189BD89B5982F917080FF3A
:1041B000FBCF8091D8008F7D8093D8008091E10063
:1041C0008F7E8093E1008091E2008F7E8093E200F9
:1041D0008091E20081608093E2008091DE03882379
:1041E00009F449C084E08093E7030E9430100E94E4
:1041F000D0068091E10083FF27C08091E20083FF19
:1042000023C08091E100877F8093E10082E080936A
:10421000E7031092DE038091E1008E7F8093E1003E
:104220008091E2008E7F8093E2008091E2008061C5
:104230008093E20042E060E080E00E94B803809159
:10424000F00088608093F000FF91EF91BF91AF91F3
:104250009F918F917F916F915F914F913F912F919E
:104260000F900FBE0F901F90189519BC1092E70386
:104270001092D10372CF8091E30087FD93E0909379
:10428000E703B3CFCDB7DEB7AA970FB6F894DEBF7A
:104290000FBECDBF84B7877F84BF0FB6F894A895B3
:1042A00080916000886180936000109260000FBE72
:1042B00080E890E00FB6F8948093610090936100DD
:1042C0000FBE85B7806885BF85B7806885BF0E94AF
:1042D000F7020E94EA038091E20084608093E2008A
:1042E00078948091E7038823A1F01091E9001F7072
:1042F0009091EC00892F817090FD80E8182B10922E
:10430000E9008091E80083FD0E943B101F7010932C
:10431000E90082E084BD93E095BD9AEF97BD80935C
:104320006E008EE090E00E94492791E0811101C06B
:1043300090E090930E010E94040D882331F061E01B
:1043400070E086E091E00E949E2580910E018091B0
:104350000E0195E0811190E09093B10385E0891BF7
:104360008093B003AAE5B1E061E070E08D91E82FA1
:10437000E295EF70F0E041A18F709B0101C0220F28
:104380008A95EAF7922F9095942391A382A1822B8C
:1043900082A321E0AF35B20749F7A4E6B1E04AE6CF
:1043A00051E061E070E08D91E82FE295EF70F0E070
:1043B00011A18F709B0101C0220F8A95EAF7922FFD
:1043C0009095912391A382A1822B82A34A175B0728
:1043D00051F7E6EAF3E0A3ECB3E011921D9283E01B
:1043E000E03BF807D1F70E948C1CEFE3FCE9319722
:1043F000F1F700C000000E948C1C8091C30380FF75
:104400000BC080E00E94B50F6FEF7FEF90E080E07F
:104410000E9485270E943A0C90E080E00E9451277C
:104420008C3E9E4F69F00E94CD0F90E080E00E948C
:1044300051278C3E9E4F21F00E94CD0F0E947B1C85
:1044400045E050E06CE170E08CEE93E00E9439278B
:104450008091EC038C7F11F40E947B1C0E94040D60
:10446000811106C061E070E086E091E00E94A52520
:1044700082E290E00E944927803209F09DC283E2E7
:1044800090E00E944927873009F096C284E290E0CC
:104490000E944927833109F08FC290E080E00E949A
:1044A00051278C3E9E4F11F00E94CD0F82E090E08C
:1044B0000E9449278093B8030E94200D9093B30374
:1044C0008093B20383E090E00E944927682F70E058
:1044D00090E080E00E94380680E191E09093B5037F
:1044E0008093B403BB24BA94222423944AEF342E3D
:1044F00050E1A52E66E9462E78E7572EECE06E2EA9
:1045000083EC93E0FAE07F2E780EA8E1CA2ED12C3E
:104510008091E703853009F46DC00E948C1C0E94D5
:10452000040D882309F4A6C0A9EBB3E0E3ECF3E0A3
:1045300010E000E0302F81912D91281709F494C0EC
:1045400090E0FF24F3942827422F4F2109F487C0DD
:1045500099A33AA38F2191E009F490E09BA30E94D4
:10456000AD048160782F9DA38CA349A15AA16BA1B2
:104570008DA10E94EF1BF801E754FC4F8081F826C3
:10458000F0820E94D0069091B703891721F00E9413
:10459000D0068093B7038091E703843009F0B8CF49
:1045A000F3E0F093E9008091E80082FFB1CF8091C1
:1045B000E80090E085FF0CC00E94160330E2E32E75
:1045C000F12C8E010F5F1F4F882309F46DC091E01D
:1045D0008091E8008B778093E800992309F498CFC5
:1045E000E981E150E33108F0A8C0F0E0EF5BF74D5E
:1045F0000C94B4268091E703843011F11092B60335
:1046000080E40FB6F894A895C09260000FBE809326
:10461000600083B7817F846083BF83B7816083BF7D
:104620007894889583B78E7F83BF0FB6F894A8954A
:1046300080916000886180936000109260000FBEDE
:104640008091DD03882309F463CF0E948C1CE3EC86
:10465000F3E0819181119BC17E12FBCF59CF9F5F07
:10466000FF0C963009F070CF0F5F1F4F0A30110515
:1046700009F060CFBEA2BFA218A60E94AD0481605F
:10468000782F9AA789A74EA15FA168A58AA50E9445
:10469000EF1B77CF8091F100F80181938F01F1E05A
:1046A000EF1AF10809F493CF8091E80085FDF2CF6D
:1046B0008091E8008B778093E8000E94160388239E
:1046C00099F385CF1A8289E08B8319C08A81823061
:1046D00009F47FC18330C1F0813079F52FB7F894A8
:1046E0006091CD037091CE038091CF039091D00360
:1046F0002FBF0E94BA266B837C838D839E83CE015D
:1047000001960E94710304CFDE011396E3ECF3E0FF
:1047100081918D9323E0ED3CF207D1F7F0CF8A81B0
:10472000823059F46B817C818D819E810E94BA26F2
:1047300085E290E00E946727E2CFB982E0CF4C810A
:104740006B818A810E942E0D9827892798279E8346
:104750008D83D5CF0D811E811027012710278A81D7
:10476000EB80E69C70011124859DE00CF11C112466
:104770008C8190E0880F991FE80EF91E612FC70108
:1047800086960E946727602FC7018796D3CF0E9425
:10479000500FB5CF8A818138D9F060F4803809F0A4
:1047A000AECF8B818093EF03873908F4A8CF409276
:1047B000EF03A5CF8238C9F0833809F0A0CF8091EC
:1047C000EF039C812B812093ED039093EE03ECCFBC
:1047D0009B8110920F01892F880F880F911103C0C0
:1047E0008093EC038CCF8160FBCF8B818093F003AF
:1047F00086CF8A81813899F030F4803809F07FCFF4
:104800008091EF0361CF823879F0833809F077CF58
:104810008091ED038B838091EE038C8370CF809128
:10482000EC038695869550CF8091F0034DCF0E9482
:10483000741365CFAA8263CF2A823B8260CFEA805D
:10484000FB80FE24EF24FE248E010F5F1F4F8C801F
:10485000800E912E911CC7018A5F9D4F0815190586
:1048600009F44DCFEAEFEE16E1E0FE0650F40E94A7
:104870004927F8018483FFEFEF1AFF0A0F5F1F4FEC
:10488000EACFF8011482F7CF0A811B811027012794
:104890001027CE0101964C01EC80E00EF12EF11CA8
:1048A000C8018A5F9D4FE016F10609F428CF0A3F40
:1048B000E1E01E0720F4F40164810E946727FFEF06
:1048C0008F1A9F0A0F5F1F4FEBCF0E94A50F17CFC4
:1048D00024E02A8314CFEA80FB80FE24EF24FE2408
:1048E0008E010F5F1F4F8C80800E912E911CC7018F
:1048F00086968016910609F402CFE0EEEE16E1E00E
:10490000FE0650F40E944927F8018483FFEFEF1A56
:10491000FF0A0F5F1F4FEBCFF8011482F7CF0A8118
:104920001B81102701271027CE0101964C01EC8036
:10493000E00EF12EF11CC80186960E151F0509F434
:10494000DECE003EE1E01E0720F4F40164810E9407
:104950006727FFEF8F1A9F0A0F5F1F4FECCF80E092
:104960000E94B50F6FEF7FEF90E080E00E948527F7
:10497000C6CECE0101960E9471032FEF81EE94E026
:10498000215080409040E1F700C0000043CDA9BC19
:1049900082E189BD09B400FEFDCF8091D8008F7DF2
:1049A0008093D8008091E00082608093E000809145
:1049B000E00081FDFCCFACCD60E085E290E00E949C
:1049C00067270E94500F0E94A50F81E00E94B50F3B
:1049D00064CD85E290E00E9449271B821C821D82E3
:1049E0008E838DCE78941F921FB61F9211248F93C1
:1049F0009F93AF93BF938091CD039091CE03A091ED
:104A0000CF03B091D0030196A11DB11D8093CD03BA
:104A10009093CE03A093CF03B093D003BF91AF91F7
:104A20009F918F911F901FBE1F9018951F921FB6C8
:104A30001F9211248F939F93AF93BF938091B603DE
:104A4000811113C08091CD039091CE03A091CF032B
:104A5000B091D0034196A11DB11D8093CD039093D9
:104A6000CE03A093CF03B093D003BF91AF919F919A
:104A70008F911F901FBE1F9018958EE14B9B02C017
:104A80008150E1F74B9BFECF08955B9880E28A95B9
:104A9000F1F75B9A0895FC013BE03A95F1F798E055
:104AA00020E080E031E040E14A95F1F7880F4B9B30
:104AB00002C08160232742E04A95F1F7000040E1FF
:104AC0004A95F1F7915079F790E19A95F1F799B1FC
:104AD00032E03A95F1F7000040E14A95F1F793FB97
:104AE000992790F992272081920F90830895EF9251
:104AF000FF920F931F93CF93DF930F92CDB7DEB743
:104B000019828C017C01E60EF11C0E151F0561F463
:104B100081E09981911180E00F90DF91CF911F91F9
:104B20000F91FF90EF9008950E943D25CE010196D0
:104B30000E944B25F80181938F01E7CF9093F603F4
:104B40008093F503539A5B9A08959093F6038093AC
:104B5000F50353985B9AEB9AE9E6F0E080818F7356
:104B6000808308956150770B91E001C0990F6A9599
:104B7000EAF720E031E0911108C0222391F05B9A1E
:104B800080E28A95F1F75B980895492F482339F020
:104B90005B9A232740E24A95F1F79695ECCF5B9814
:104BA000F9CF5B98EDCFFF920F931F93CF93DF93D5
:104BB000EC018C01060F111DC017D10731F4DF91F4
:104BC000CF911F910F91FF900895F9900E94452574
:104BD00068E08F2D0E94B225EFCF1F920F920FB683
:104BE0000F9211242F933F934F935F936F937F9373
:104BF0008F939F93AF93BF93CF93DF93EF93FF93E5
:104C00005B98539AC091F503D091F6036D816623AA
:104C100021F08E819F810E94D3250E94452580E14D
:104C20008A95F1F75B9853985B9A80E18A95F1F742
:104C30006A81662309F18B819C810E947725E88136
:104C4000F981882311F088E001C082E080830E940E
:104C50003D25FF91EF91DF91CF91BF91AF919F9152
:104C60008F917F916F915F914F913F912F910F9015
:104C70000FBE0F901F901895E881F981E4CFCF9374
:104C8000DF93C091F503D091F603F894539A5B98A3
:104C900085E08A95F1F7000053985B9A80E28A9547
:104CA000F1F74B9B0CC0539A5B9AE881F98181E044
:104CB0008083789481E090E0DF91CF9108956D81B9
:104CC000662381F08E819F810E94772581110AC021
:104CD000539A5B9AE881F98182E08083789482E03C
:104CE00090E0EACF0E943D2580E28A95F1F75B983B
:104CF000539A80E18A95F1F76A81662321F08B81CE
:104D00009C810E94D3250E944525E881F98110826B
:104D1000789490E080E0D0CFAA1BBB1B51E107C084
:104D2000AA1FBB1FA617B70710F0A61BB70B881F3B
:104D3000991F5A95A9F780959095BC01CD010895CA
:104D400097FB072E16F4009407D077FD09D00E9438
:104D50008C2607FC05D03EF4909581959F4F0895D1
:104D6000709561957F4F0895EE0FFF1F0590F491A8
:104D7000E02D0994692796276927782787277827C0
:104D80000895CF92DF92EF92FF92CF93DF93CDB74A
:104D9000DEB72A970FB6F894DEBF0FBECDBF898766
:104DA0009A87A985BA852D913D914D915C91298372
:104DB0003A834B835C83232B242B252B41F424E261
:104DC00039ED4BE557E029833A834B835C83698156
:104DD0007A818B819C812DE133EF41E050E00E948C
:104DE0008B2769017A01A7EAB1E49B01AC010E941B
:104DF000AA2769837A838B839C83ACEEB4EFA701E7
:104E000096010E94B8279B01AC0189819A81AB81F0
:104E1000BC81820F931FA41FB51FB7FF03C001976A
:104E2000A109B048E985FA8580839183A283B38381
:104E30009F772A960FB6F894DEBF0FBECDBFDF91E5
:104E4000CF91FF90EF90DF90CF9008950E94C12600
:104E5000089580E091E00E94C1260895B0E0A0E0AE
:104E60008093000190930101A0930201B09303018C
:104E70000895DC01CB01FC01F999FECF06C0F2BD1B
:104E8000E1BDF89A319600B40D9241505040B8F708
:104E90000895F999FECF92BD81BDF89A992780B502
:104EA0000895A8E1B0E042E050E00C943B27DC011B
:104EB000A40FB51F4150504048F0CB01840F951FFF
:104EC0002E910E94682741505040D0F70895262F18
:104ED000F999FECF92BD81BDF89A019700B40216F0
:104EE00039F01FBA20BD0FB6F894FA9AF99A0FBE9E
:104EF00008950396272F0E9468270E946727252F71
:104F00000E946827242F0C9468270196272F0E945F
:104F100068270C946727052E97FB1EF400940E94C7
:104F2000A22757FD07D00E94BD2707FC03D04EF4EF
:104F30000C94A22750954095309521953F4F4F4FA7
:104F40005F4F089590958095709561957F4F8F4F35
:104F50009F4F08950E94DF27A59F900DB49F900D4D
:104F6000A49F800D911D11240895B7FF0C94AA27CA
:104F70000E94AA27821B930B0895A1E21A2EAA1B56
:104F8000BB1BFD010DC0AA1FBB1FEE1FFF1FA217F9
:104F9000B307E407F50720F0A21BB30BE40BF50BF6
:104FA000661F771F881F991F1A9469F7609570957F
:104FB000809590959B01AC01BD01CF010895A29F02
:104FC000B001B39FC001A39F700D811D1124911DDD
:104FD000B29F700D811D1124911D0895F894FFCF8B
:104FE0003B0F3B0F440F440F460F440F440F440F39
:104FF0003B0F3B0F4B0F440F440F4B0F2011481139
:10500000F4124811F4127B119C11F412A512B21281
:10501000AF16BA16C116C616CB16D016D516DA16A6
:10502000DF16E416E916EE16F316F816FD164F1401
:105030004F144F144F144F1417171717881788174A
:10504000DF174D174D174D17FB17DD18EC18EC182F
:10505000C11DCB1D0F1E551E9C1EE21E2B1F311F96
:10506000341F391F3C1F411F441F471F4A1F4D1F3C
:10507000501F531F561F591F5C1F611F641F671F5E
:10508000A91F622366238F239F23AA23C723CA2332
:10509000F9231724AF24B9241A241C241F244424E0
:0850A000652468246B248F24B1
:1050A80001000000FFFF7202007202057A0201038C
:1050B800AA04090CA904050CFC0B0100FF0000FF61
:1050C80096003131295A1B750A818283E200E90072
:1050D800EA00B500B600B700CD008301CC008A0114
:1050E80092019401210223022402250226022702AA
:1050F8002A02B300B4006F007000F1F5F7353400F0
:1051080000000000F4F6676636944022320001DEA3
:1051180000AC00D204EB040B0500010203040506F1
:105128000708090A0B0C0D0E0F101112131415168F
:105138001718191A1B1C1D1E1F202122232425267F
:105148002728292A2B2C2D2E2F303132333435366F
:105158003738393A3B660051003D002900140000F9
:1051680000661051103D10291014100010662051CF
:10517800203D20292014200020663051303D302960
:105188003014300030664051403D40294014400002
:1051980040E000CC00B700A3008F007A00E010CCFC
:1051A80010B710A3108F107A10E020CC20B720A3DE
:1051B800208F207A20E030CC30B730A3308F307A7F
:1051C80030E040CC40B740A3408F407A400404040C
:1051D8000404010404040404010404040404010490
:1051E800040404040101010101010101040404048F
:1051F8000401040404040401040404040401040470
:0A520800040404010101010101008A
:00000001FF
